:100000000C946F010C9497010C9497010C94970138
:100010000C9497010C9497010C9497010C94970100
:100020000C9497010C9497010C94D6060C949D05A2
:100030000C9497010C9497010C9497010C949701E0
:100040000C9497010C9497010C9497010C949701D0
:100050000C9497010C9497010C9497010C94210235
:100060000C9497010C9497010C9497010C949701B0
:100070000C9497010C9497010C9497010C949701A0
:100080000C9497010C9497010C9497010C94970190
:100090000C9497010C9497010C9497010C94970180
:1000A0000C9497010C9497010C94970100000000A8
:1000B000240027002A002D00300000000000250049
:1000C00028002B002E003100000000002300260035
:1000D00029002C002F000404040404030405020278
:1000E00002020403020202020606060606060404D1
:1000F00002020204040802011040804010204080E7
:10010000408008020401804020100201108010206D
:1001100040400000000200080E0000030401000B34
:1001200000000000070605040100080A0B0C0D0979
:100130000403090422034100720064007500690091
:100140006E006F0020004C0065006F006E006100C3
:10015000720064006F0018034100720064007500B3
:1001600069006E006F0020004C004C00430012013B
:1001700000020000004041233400000101020001A0
:10018000120100020200004041233400000101027C
:10019000000100C18081C105010902A1010901A17D
:1001A000008501050919012903150025019503752D
:1001B00001810295017505810305010930093109A5
:1001C000381581257F750895038106C0C005010992
:1001D00006A1018502050719E029E715002501752B
:1001E000019508810295017508810395067508152A
:1001F0000025650507190029658100C00904020072
:10020000010300000009210101000122650007052A
:10021000840340000100000000000000002A2B2899
:1002200000000000000000000000000000000000CE
:1002300000000000002C9EB4A0A1A2A434A6A7A593
:10024000AE362D3738271E1F20212223242526B322
:1002500033B62EB7B89F8485868788898A8B8C8D24
:100260008E8F909192939495969798999A9B9C9D36
:100270002F3130A3AD350405060708090A0B0C0D14
:100280000E0F101112131415161718191A1B1C1D16
:10029000AFB1B0B500080B00020202010009040072
:1002A00000010202000005240010010524010101E3
:1002B00004240206052406000107058103100040FE
:1002C00009040100020A00000007050202400000C4
:1002D000070583024000000047073B08020911247C
:1002E0001FBECFEFDAE0DEBFCDBF11E0A0E0B1E08E
:1002F000E2E4F2E102C005900D92A233B107D9F712
:1003000011E0A2E3B1E001C01D92AD35B107E1F704
:1003100012E0CEEDD2E004C02297FE010E941B093C
:10032000C83DD107C9F70E94BC030C941F090C9467
:1003300000001F93CF93DF9383EF80BB81BB82E1EB
:1003400061E00E9484038BE491E060E071E00E9430
:100350008307C5E28C2F61E00E946003C150D0F793
:10036000CBE0D0E01AC015E2812F61E00E94840347
:100370001150D0F767E070E080E090E00E948F02BB
:1003800015E2812F60E00E9484031150D0F763E0F2
:1003900070E080E090E00E948F02219721F7DF91CA
:1003A000CF911F910895809134019091350186324B
:1003B000910581F4809132019091330121E030E088
:1003C0008227932790933301809332011092350155
:1003D0001092340180913601909137019C012F5F7A
:1003E0003F4F30933701209336018333910564F0FA
:1003F00081E090E090933701809336018BE491E0A7
:1004000060E071E00E948307809134019091350192
:100410009C012F5F3F4F309335012093340161E001
:1004200020913201309133012115310509F060E04E
:100430000E9484036AE070E080E090E00E948F02F6
:1004400008951F920F920FB60F9211242F933F938E
:100450008F939F93AF93BF9380913C0190913D0107
:10046000A0913E01B0913F01309140010196A11D44
:10047000B11D232F2D5F2D3720F02D570196A11D83
:10048000B11D2093400180933C0190933D01A093C6
:100490003E01B0933F018091380190913901A091C4
:1004A0003A01B0913B010196A11DB11D8093380125
:1004B00090933901A0933A01B0933B01BF91AF9162
:1004C0009F918F913F912F910F900FBE0F901F9092
:1004D00018959FB7F89420913801309139014091D7
:1004E0003A0150913B0186B5A89B06C08F3F21F091
:1004F0002F5F3F4F4F4F5F4F9FBF542F432F322FE0
:100500002227280F311D411D511D82E0220F331F6C
:10051000441F551F8A95D1F7B901CA010895EF927A
:10052000FF920F931F93CF93DF937B018C010E9467
:100530006902EB010FC00E9469026C1B7D0B83E016
:10054000683E780738F00894E108F10801091109BC
:10055000C851DC4FE114F1040105110561F7DF9189
:10056000CF911F910F91FF90EF900895789484B5EB
:10057000826084BD84B5816084BD85B5826085BD9F
:1005800085B5816085BDEEE6F0E080818160808385
:10059000E1E8F0E010828081826080838081816068
:1005A0008083E0E8F0E0808181608083E1EBF0E02F
:1005B000808184608083E0EBF0E0808181608083D3
:1005C000E1E9F0E0808182608083808181608083C6
:1005D000E0E9F0E0808181608083E1ECF0E08081FF
:1005E00082608083808181608083E0ECF0E08081A4
:1005F00081608083EAE7F0E080818460808380818D
:100600008260808380818160808380818068808334
:1006100008958730A9F1883080F48330E1F0843088
:1006200030F4813011F1823009F049C021C08430AA
:10063000B1F0863009F043C01FC08A3079F18B30A9
:1006400028F4883019F18930D1F524C08B3061F15C
:100650008C30A9F52FC0809180008F7703C08091E6
:1006600080008F7D80938000089584B58F7702C0CD
:1006700084B58F7D84BD08958091B0008F7703C0CD
:100680008091B0008F7D8093B0000895809190009C
:100690008F7707C0809190008F7D03C0809190007C
:1006A000877F8093900008958091C0008F7780931A
:1006B000C00008958091C0008F7D8093C000089590
:1006C00090E0FC01EC50FF4F2491FC01EA52FF4FF7
:1006D000E491EE23C1F0F0E0EE0FFF1FE455FF4F71
:1006E00085919491DC01662341F49FB7F8948C9135
:1006F000209582238C939FBF08959FB7F8948C9187
:10070000822B8C939FBF08950F931F93DF93CF93FA
:100710000F92CDB7DEB7282F30E0F901EE5EFE4F25
:100720008491F901EC50FF4F14912A523F4FF90187
:1007300004910023D9F0882321F069830E940903E2
:100740006981E02FF0E0EE0FFF1FE654FF4F859127
:100750009491DC019FB7F894662321F48C91109555
:10076000812302C08C91812B8C939FBF0F90CF91DE
:10077000DF911F910F910895CF93DF930E94B602EE
:1007800089E491E00E942E070E949901C0E0D0E028
:100790000E94D3012097E1F30E940000F9CF8091DD
:1007A000E80080FFFCCF0895FC0104C08091F100B7
:1007B000819361506623D1F7289884E680934201A3
:1007C00008952FB7FC012083F89467706093E900C7
:1007D0000895DF93CF930F92CDB7DEB7682FCE0188
:1007E00001960E94E1038091F20099819FBF0F90D2
:1007F000CF91DF910895FF920F931F93DF93CF93D3
:1008000000D0CDB7DEB7282FF62E8A0180914301A4
:100810008823C9F057FF22C016C0289820934201B0
:100820003091F1003193E817F907B9F70115110577
:1008300039F08091F200882319F48BE68093E80068
:1008400089818FBF02C00FEF1FEFC8010F900F907B
:10085000CF91DF911F910F91FF900895CE010196E6
:10086000622F7A830E94E1038091F20090E07A8106
:10087000801791070CF48C01EF2DF72FCF01800F1B
:10088000911D24E6D0CFDF93CF930F92CDB7DEB783
:10089000BE016F5F7F4F41E050E00E94FB0381305B
:1008A000910519F4298130E002C02FEF3FEFC90113
:1008B0000F90CF91DF910895DF93CF930F92CDB733
:1008C000DEB7682FCE0101960E94E1038091E80017
:1008D00085FF05C09091F20080E4891B01C080E093
:1008E00099819FBF0F90CF91DF9108952F923F92F2
:1008F0004F925F926F927F928F929F92AF92BF9230
:10090000CF92DF92EF92FF920F931F93DF93CF93DB
:100910000F92CDB7DEB7D82EC42EA52E80914301FD
:10092000882309F46FC0062F172FE42EF52E2AEF27
:10093000B22E3E010894611C711C2D2C332490E2D0
:10094000492E512C422053208AE3882E80E428220D
:1009500033244DC08D2D0E945C04982E882351F4C1
:10096000BA9409F44FC061E070E080E090E00E942A
:100970008F023DC090E0E816F9060CF49E2CE918B1
:10098000F108C3016D2D0E94E1034114510439F0B7
:1009900003C01092F1009A949920D9F71AC0D7FC9D
:1009A00003C0892DF80111C0892D980107C0F901F4
:1009B0002F5F3F4FE491E093F10081508823B9F716
:1009C00006C091919093F10081508823D1F7090DD1
:1009D000111D8091E80085FF06C0E114F10429F49F
:1009E0002114310411F08092E80089818FBFE11455
:1009F000F10409F0AFCF5D9884E6809341012C2D7E
:100A00003A2D02C02FEF3FEFC9010F90CF91DF9138
:100A10001F910F91FF90EF90DF90CF90BF90AF901C
:100A20009F908F907F906F905F904F903F902F900E
:100A300008951092E900109245011092440190939C
:100A40004701809346010895CF93242F352FE62F39
:100A5000F72F9EEF34C087FF02C0C49101C0C08150
:100A6000A0914401B0914501609146017091470108
:100A7000A617B707BCF46091E8006570E1F36091D8
:100A8000E80062FD22C0C093F100609144017091C2
:100A900045016F5F7F4F6F7370706115710511F4C1
:100AA0009093E80060914401709145016F5F7F4F22
:100AB00070934501609344012150304031962115D7
:100AC000310549F6242F352F02C02FEF3FEFC90122
:100AD000CF9108951F93DF93CF930F92CDB7DEB7D9
:100AE000162F2091E80022FFFCCF612F79830E940E
:100AF000D4038BEF8093E800812F7981972F0F909B
:100B0000CF91DF911F9108950F931F93DF93CF93A0
:100B10000F92CDB7DEB719828E010F5F1F4FC8014C
:100B20000E94B908C8010E948607898190E00F9051
:100B3000CF91DF911F910F9108951F920F920FB6E1
:100B40000F921124EF92FF920F931F932F933F93D5
:100B50004F935F936F937F938F939F93AF93BF93C5
:100B6000EF93FF93DF93CF93CDB7DEB76297DEBFEE
:100B7000CDBF1092E9008091E80083FFF3C0CE0161
:100B8000019668E00E94D40382EF8093E800098117
:100B900007FF03C00E94CF0303C08EEF8093E800DD
:100BA000802F90E09C01207630702115310509F0EE
:100BB000BEC02A81222329F41092F1001092F10084
:100BC000CAC0213009F4C7C0233009F4C4C025309D
:100BD00039F40E94CF038B8180688093E300BBC00F
:100BE000263009F076C02C810F811885223081F5DE
:100BF00080E090E02A8B0E9419050E94840599E00C
:100C000039E0E32EF12CEC0EFD1EF701392F119285
:100C10003A95E9F799872A892A8791E09E8790E893
:100C2000988B9AEF998B2091440130914501275F71
:100C30003F4F3C872B878D87C8010E94190580E0B4
:100C4000B70149E050E00E9424050E94840583C05A
:100C5000C8012A8B0E9419052A89223241F482E2B6
:100C600090E00E949207009709F075C078C021308B
:100C700079F48F8198858830910519F481E080930B
:100C80004801809148018823B9F060E871E016C0FE
:100C9000233009F064C08B81882319F460E371E08C
:100CA0000DC0823019F464E371E008C0813009F0AE
:100CB00056C066E571E002C06EE671E0611571052F
:100CC00009F44DC0FB01449180E850E00E942405E6
:100CD00042C0273009F443C0283021F481E08093DA
:100CE000F10039C02930B9F5837090700097B9F5DB
:100CF00080E090E031E026E3482F4F5F4093E90029
:100D00003093EB000196FC01EE56FE4FE491E09328
:100D1000EC002093ED008430910571F78EE780930D
:100D2000EA001092EA008B818093430114C08F8106
:100D300098850E9419058D81882329F4CE0101969A
:100D40000E94C50806C0823051F4CE0101960E946F
:100D5000BB07882321F08EEF8093E80003C081E277
:100D60008093EB006296DEBFCDBFCF91DF91FF9104
:100D7000EF91BF91AF919F918F917F916F915F9113
:100D80004F913F912F911F910F91FF90EF900F90F6
:100D90000FBE0F901F9018958093E9008091F2008C
:100DA000882319F08AE38093E80008951F920F9238
:100DB0000FB60F9211242F933F934F935F936F932E
:100DC0007F938F939F93AF93BF93EF93FF93809104
:100DD000E1001092E10083FF0FC01092E90091E062
:100DE0009093EB001092EC0092E39093ED00109240
:100DF000430198E09093F00082FF1FC083E00E94BF
:100E0000CC0680914101882351F0809141018150AD
:100E10008093410180914101882309F45D9A80917A
:100E20004201882351F08091420181508093420118
:100E300080914201882309F4289AFF91EF91BF9194
:100E4000AF919F918F917F916F915F914F913F9162
:100E50002F910F900FBE0F901F9018951092430185
:100E600081E08093D70080EA8093D80082E189BD39
:100E700089B580FFFDCF80E98093D8008CE0809316
:100E8000E2001092E000559A209A0895089508957E
:100E9000CF92DF92EF92FF920F931F93CF93DF9346
:100EA0006C017B018A01C0E0D0E00FC0D7016D91D9
:100EB0007D01D601ED91FC910190F081E02DC601FC
:100EC0000995C80FD91F015010400115110571F780
:100ED000CE01DF91CF911F910F91FF90EF90DF90A6
:100EE000CF900895DB010D900020E9F7AD0141504E
:100EF0005040461B570BDC01ED91FC910280F381C1
:100F0000E02D099508950E9472070895FC018081E3
:100F10008F5F808380E86CEF71E049E150E00E94D0
:100F20002405089580E867E971E045E650E00E94F5
:100F300024050895EF92FF920F931F93DF93CF93B1
:100F40000F92CDB7DEB789838B017A0184E0BE01B1
:100F50006F5F7F4F41E050E00E94760484E4B80167
:100F6000A7010E9476040F90CF91DF911F910F91FE
:100F7000FF90EF900895FC0191818081813A31F4D6
:100F8000913089F081E0933081F412C0813269F4AC
:100F90009B3021F4828180930E0105C09A3039F490
:100FA000828180930F0181E0089580E0089580E0C0
:100FB000089582E048E050E00E949A070895EF9279
:100FC000FF920F931F93DF93CF93CDB7DEB7289790
:100FD0000FB6F894DEBF0FBECDBF8C01AE014F5FE0
:100FE0005F4F88E0FA0111928A95E9F7F801848150
:100FF0009581009741F0FC01A081B181ED91FC91B8
:1010000070E0099517C067FD07C0E62FF0E0EB5EC2
:10101000FD4FE491EE2341F481E090E0F8019383E9
:10102000828320E030E019C0E7FF03C082E08983BB
:10103000EF77EB83C8017E010894E11CF11CB70136
:101040000E94D90788E0F70111928A95E9F7C80153
:10105000B7010E94D90721E030E0C90128960FB6F8
:10106000F894DEBF0FBECDBFCF91DF911F910F91DE
:10107000FF90EF90089510924A0110924E01109245
:101080004D01EDE4F1E08EE191E0929382931582BF
:101090001482089520911001309111014FEF2F3FDC
:1010A000340759F4DC01ED91FC910680F781E02DC5
:1010B00009959093110180931001809110019091F6
:1010C000110108950F931F93DF93CF930F92CDB724
:1010D000DEB78C01698380911901882369F083E070
:1010E000BE016F5F7F4F41E050E00E94760418160A
:1010F000190614F49C0107C081E090E0F801938385
:10110000828320E030E0C9010F90CF91DF911F91E1
:101110000F91089583E00E94CC060895209110015C
:10112000309111018FEF2F3F380739F08FEF9FEF8C
:10113000909311018093100104C082E00E94430447
:101140009C01C901089582E00E94E90320911001E9
:10115000309111019FEF2F3F390709F08F5F90E029
:10116000089589E491E00E944607F8940C94003CAD
:101170000895FC0180818E5F808380E865E972E0DC
:1011800042E450E00E9424050895CF93DF93EC01E0
:1011900089819881913A51F4813281F580E062E150
:1011A00071E047E050E00E94240526C0913231F5FD
:1011B000803239F482E191E067E070E00E946A05D4
:1011C0001BC08232D9F480911901882391F02091BB
:1011D0001201309113014091140150911501203BEF
:1011E00084E0380780E0480780E0580711F40E9447
:1011F000B1088A818093190181E001C080E0DF910C
:10120000CF910895109254011092530188EE93E00B
:10121000A0E0B0E08093550190935601A093570150
:10122000B093580186E291E090935201809351016E
:101230000895EE0FFF1F0590F491E02D0994F894A6
:02124000FFCFDE
:1012420048656C6C6F2041726475696E6F000101B4
:10125200FFFF00E100000000000000000000DF07C7
:1012620048070000000062084807A3088E084A08E1
:021272008A08E8
:00000001FF
